:020000040000FA
:040800004BEF04F0C6
:1008100003B20EEF04F08B7429EF04F0039203018E
:1008200003EE00F080517F0BE92604C0EFFF802B20
:100830008151805D700BD8A48B8200008051815D56
:10084000700BD8A48B9281518019D8B4079029EFEE
:1008500004F002C0E0FF005001C0D8FF1000A6B2B3
:100860002FEF04F00CC0A9FF0BC0A8FFA69EA69C0A
:10087000A684F29E550EA76EAA0EA76EA682F28ED1
:10088000A694A6B241EF04F01200A96EA69EA69C03
:10089000A680A8501200076A0E6A0F6A0F010E0E9A
:1008A000C16E860EC06E030EC26E0F01600E896EA1
:1008B000110E926E0E0E8A6EE10E936E8B6A800E92
:1008C000946EF18EF29A9D909D92FF0ECB6E200E4B
:1008D000BB6E0C0EBA6E760ECA6EE6EC09F0160E02
:1008E00045EC04F0E8CF00F1170E45EC04F0E8CF3A
:1008F00001F1180E45EC04F0E8CF02F1190E45ECB9
:1009000004F0E8CF03F1010103AFA1EF04F079ECAB
:1009100009F0160E0C6E00C10BF02FEC04F0170E50
:100920000C6E01C10BF02FEC04F0180E0C6E02C11E
:100930000BF02FEC04F0190E0C6E03C10BF02FEC32
:1009400004F000C15DF101C15EF102C15FF103C1BC
:1009500060F100C161F101C162F102C163F103C143
:1009600064F11A0E45EC04F0E8CF00F11B0E45ECE3
:1009700004F0E8CF01F11C0E45EC04F0E8CF02F1E1
:100980001D0E45EC04F0E8CF03F1010103AFF7EFD2
:1009900004F079EC09F01A0E0C6E00C10BF02FEC8C
:1009A00004F01B0E0C6E01C10BF02FEC04F01C0EBA
:1009B0000C6E02C10BF02FEC04F01D0E0C6E03C187
:1009C0000BF02FEC04F01A0E45EC04F0E8CF00F128
:1009D0001B0E45EC04F0E8CF01F11C0E45EC04F0D1
:1009E000E8CF02F11D0E45EC04F0E8CF03F100C1A1
:1009F00065F101C166F102C167F103C168F1240E1E
:100A0000AC6E900EAB6E240EAC6E080EB86E000E7F
:100A1000B06E1F0EAF6E0401806B816B0F01900EE4
:100A2000AB6E0F019D8A0301806B816BA26B8B9271
:100A300007900001F28EF28C07B004EF07F003017B
:100A4000805181197F0BD8B404EF07F013EE00F04A
:100A500081517F0BE126812BE7CFE8FFE00BD8B473
:100A600004EF07F023EE82F0A2511F0BD926E7CF47
:100A7000DFFFA22BDF50780AD8A404EF07F007802D
:100A800061C100F162C101F163C102F164C103F10E
:100A90000101040E046F000E056F000E066F000EBC
:100AA000076F82EC08F000AF5FEF05F00101030E65
:100AB000616F000E626F000E636F000E646F0301C2
:100AC0008251690AD8B4ECEF05F08251760AD8B4A5
:100AD00084EF05F08251560AD8B4B3EF05F0FFEF6A
:100AE00006F0040114EE00F080517F0BE12682C471
:100AF000E7FF802B12000D0E826F71EC05F00A0EDD
:100B0000826F71EC05F01200BAEC09F083C324F196
:100B100084C325F185C326F186C327F10101C7EC03
:100B200009F03EEC09F000C10CF101C10DF102C168
:100B30000EF103C10FF1D8900333023301330033B8
:100B4000D89003330233013300330C470C470C4772
:100B50000C47300E0C170C0E0C1300C1BBFF0CC160
:100B6000BAFFFFEF06F0BAEC09F083C324F184C3A7
:100B700025F185C326F186C327F1C7EC09F03EECC9
:100B800009F027EC0AF0BAEC09F088C324F189C314
:100B900025F18AC326F18BC327F1C7EC09F03EEC9F
:100BA00009F05AEC0AF0BAEC09F08DC324F18EC3B7
:100BB00025F18FC326F190C327F1C7EC09F03EEC75
:100BC00009F08DEC0AF00401760E826F71EC05F0ED
:100BD0007BEC05F0FFEF06F00401690E826F71EC0B
:100BE00005F004012C0E826F71EC05F00101040E7A
:100BF000006F000E016F000E026F000E036F1CEC01
:100C000009F020C182F40401300E822771EC05F056
:100C100021C182F40401300E822771EC05F022C15B
:100C200082F40401300E822771EC05F023C182F4B6
:100C30000401300E822771EC05F024C182F4040116
:100C4000300E822771EC05F025C182F40401300ECC
:100C5000822771EC05F026C182F40401300E822750
:100C600071EC05F027C182F40401300E822771EC8B
:100C700005F004012C0E826F71EC05F001010A0EE3
:100C8000006F000E016F000E026F000E036F1CEC70
:100C900009F020C182F40401300E822771EC05F0C6
:100CA00021C182F40401300E822771EC05F022C1CB
:100CB00082F40401300E822771EC05F023C182F426
:100CC0000401300E822771EC05F024C182F4040186
:100CD000300E822771EC05F025C182F40401300E3C
:100CE000822771EC05F026C182F40401300E8227C0
:100CF00071EC05F027C182F40401300E822771ECFB
:100D000005F004012C0E826F71EC05F00101130E49
:100D1000006F000E016F000E026F000E036F1CECDF
:100D200009F020C182F40401300E822771EC05F035
:100D300021C182F40401300E822771EC05F022C13A
:100D400082F40401300E822771EC05F023C182F495
:100D50000401300E822771EC05F024C182F40401F5
:100D6000300E822771EC05F025C182F40401300EAB
:100D7000822771EC05F026C182F40401300E82272F
:100D800071EC05F027C182F40401300E822771EC6A
:100D900005F004012C0E826F71EC05F0200EF86E48
:100DA000F76AF66A04010900F5CF82F471EC05F0E8
:100DB0000900F5CF82F471EC05F00900F5CF82F45B
:100DC00071EC05F00900F5CF82F471EC05F0090033
:100DD000F5CF82F471EC05F00900F5CF82F471ECE7
:100DE00005F00900F5CF82F471EC05F00900F5CFAC
:100DF00082F471EC05F07BEC05F0FFEF06F00301E7
:100E0000A26B079004EF07F00401805181197F0B5A
:100E10000BE09EA809D014EE00F081517F0BE12673
:100E2000E750812B0F01AD6E1CEF05F00CC100F1F6
:100E30000DC101F10EC102F10FC103F1000E046FEB
:100E4000000E056F010E066F000E076FB0EC08F084
:100E50001DA141EF07F01451D8B441EF07F00CC1C8
:100E600000F10DC101F10EC102F10FC103F1000E3D
:100E7000046F000E056F0A0E066F000E076FB0ECD0
:100E800008F0120001010C6B0D6B0E6B0F6B120062
:100E90001EC182F40401300E822771EC05F01FC1DF
:100EA00082F40401300E822771EC05F020C182F437
:100EB0000401300E822771EC05F021C182F4040197
:100EC000300E822771EC05F022C182F40401300E4D
:100ED000822771EC05F023C182F40401300E8227D1
:100EE00071EC05F024C182F40401300E822771EC0C
:100EF00005F025C182F40401300E822771EC05F063
:100F000026C182F40401300E822771EC05F027C15E
:100F100082F40401300E822771EC05F01200010109
:100F2000005305E1015303E1025301E1002B52ECB0
:100F300008F079EC09F02C51006F2D51016F420E31
:100F4000046F4B0E056F000E066F000E076F91ECDD
:100F500008F000C104F101C105F102C106F103C1AD
:100F600007F10CC100F10DC101F10EC102F10FC179
:100F700003F107B2C0EF07F086EC08F0C2EF07F00C
:100F800082EC08F000C10CF101C10DF102C10EF1BB
:100F900003C10FF1120079EC09F04CC100F14DC111
:100FA00001F1060E45EC04F0E8CF04F1070E45EC24
:100FB00004F0E8CF05F1080E45EC04F0E8CF06F1A7
:100FC000090E45EC04F0E8CF07F182EC08F000C10F
:100FD00018F101C119F102C11AF103C11BF1290E67
:100FE000046F000E056F000E066F000E076F91EC88
:100FF00008F0EE0E046F430E056F000E066F000E34
:10100000076F86EC08F018C104F119C105F11AC187
:1010100006F11BC107F191EC08F000C110F101C10C
:1010200011F102C112F103C113F1120E45EC04F0EB
:10103000E8CF04F1130E45EC04F0E8CF05F1140EEF
:1010400045EC04F0E8CF06F1150E45EC04F0E8CFCE
:1010500007F10D0E006F000E016F000E026F000E03
:10106000036F91EC08F0180E046F000E056F000E70
:10107000066F000E076FB0EC08F010C104F111C14B
:1010800005F112C106F113C107F186EC08F06A0EF2
:10109000046F2A0E056F000E066F000E076F82ECBC
:1010A00008F01200BF0EFA6E200E2D6F2C6BD89038
:1010B0000037013702370337D8B063EF08F02D2F20
:1010C00058EF08F02C072D070353D8B41200033152
:1010D000070B8009326F03390F0B010F2C6F80EC67
:1010E0005FF0336F2C0580EC5FF0335D335F2C6B6A
:1010F0003233D8B02C272C3332A978EF08F0335193
:101100002C2712009EEC09F0D8B0120003510719E9
:10111000286F61EC09F0D8900751031928AF800FB0
:101120001200286B85EC09F0D8A09BEC09F0D8B030
:10113000120070EC09F079EC09F01F0E296FB1EC88
:1011400009F00B35D8B061EC09F0D8A00335D8B060
:101150001200292F9FEF08F028B188EC09F0120047
:10116000286B04510511061107110008D8A085EC61
:1011700009F0D8A09BEC09F0D8B01200086B096BFD
:101180000A6B0B6BB1EC09F01F0E296FB1EC09F083
:1011900007510B5DD8A4D9EF08F006510A5DD8A419
:1011A000D9EF08F00551095DD8A4D9EF08F0045132
:1011B000085DD8A0ECEF08F00451085F0551D8A0F5
:1011C000053D095F0651D8A0063D0A5F0751D8A02A
:1011D000073D0B5FD8900081292FC6EF08F028B19A
:1011E00088EC09F0286B85EC09F0D890B5EC09F093
:1011F00007510B5DD8A409EF09F006510A5DD8A488
:1012000009EF09F00551095DD8A409EF09F004516F
:10121000085DD8A018EF09F0003F18EF09F0013F72
:1012200018EF09F0023F18EF09F0032BD8B41200B1
:1012300028B188EC09F012000101286B85EC09F057
:10124000D8B01200BAEC09F0200E296F0037013730
:101250000237033711EE27F00A0E2A6FE7360A0E1F
:10126000E75CD8B0E76EE5522A2F2EEF09F0292F60
:1012700026EF09F028B11D81D890120001010A0E55
:10128000286F200E296F11EE1DF028512A6F0A0ECB
:10129000D890E652D8B0E726E7322A2F49EF09F076
:1012A0000333023301330033292F43EF09F0E750B2
:1012B000FF0FD8A00335D8B012001DB188EC09F09B
:1012C0001200045100270551D8B0053D01270651F1
:1012D000D8B0063D02270751D8B0073D03271200BA
:1012E0000051086F0151096F02510A6F03510B6FD2
:1012F00012000101006B016B026B036B1200010114
:10130000046B056B066B076B12000335D8A0120047
:101310000351800B001F011F021F031F003F98EFA6
:1013200009F0013F98EF09F0023F98EF09F0032B15
:10133000282B032512000735D8A012000751800B77
:10134000041F051F061F071F043FAEEF09F0053FEE
:10135000AEEF09F0063FAEEF09F0072B282B07256B
:1013600012000037013702370337083709370A37C9
:101370000B37120001011D6B1E6B1F6B206B216B65
:10138000226B236B246B256B266B276B12001E517F
:101390000F0B1E6F1F510F0B1F6F20510F0B206F74
:1013A00021510F0B216F22510F0B226F23510F0B75
:1013B000236F24510F0B246F25510F0B256F2651DE
:1013C0000F0B266F27510F0B276F1200400EC76EB1
:1013D000200EC66E81929E96C69E300EC96EFF0E7E
:1013E0009EB602D0E82EFCD79E96C69E640EC96EAD
:1013F000FF0E9EB602D0E82EFCD7818281929E9687
:10140000C69EB00EC96EFF0E9EB602D0E82EFCD767
:101410009E96C69E640EC96EFF0E9EB602D0E82E42
:10142000FCD7818281949E96C69E300EC96EFF0EB7
:101430009EB602D0E82EFCD79E96C69E640EC96E5C
:10144000FF0E9EB602D0E82EFCD781841200400E1B
:10145000C76E200EC66E819201C1E8FF30099E96CC
:10146000C69EE8CFC9FFFF0E9EB602D0E82EFCD77D
:101470009E96C69E00C1C9FFFF0E9EB602D0E82E02
:10148000FCD78182819201C1E8FFB0099E96C69E79
:10149000E8CFC9FFFF0E9EB602D0E82EFCD79E967D
:1014A000C69E00C1C9FFFF0E9EB602D0E82EFCD733
:1014B00081821200400EC76E200EC66E819401C15B
:1014C000E8FF30099E96C69EE8CFC9FFFF0E9EB684
:1014D00002D0E82EFCD79E96C69E00C1C9FFFF0E23
:1014E0009EB602D0E82EFCD78184819401C1E8FF2A
:1014F000B0099E96C69EE8CFC9FFFF0E9EB602D0E9
:10150000E82EFCD79E96C69E00C1C9FFFF0E9EB670
:1015100002D0E82EFCD781841200400EC76E200E48
:10152000C66E809C01C1E8FF30099E96C69EE8CF3A
:10153000C9FFFF0E9EB602D0E82EFCD79E96C69E2F
:1015400000C1C9FFFF0E9EB602D0E82EFCD7808CEA
:10155000809C01C1E8FFB0099E96C69EE8CFC9FFF6
:10156000FF0E9EB602D0E82EFCD79E96C69E00C106
:10157000C9FFFF0E9EB602D0E82EFCD7808C809A61
:04158000808A12004B
:10BF0000E844F926000C160C2B0C3F0C520C640C68
:10BF1000760C860C960CA50CB30CC10CCF0CDC0C6B
:06BF2000E80CF40C000C1B
:00000001FF
